:04000000D0EF03F04A
:0800080000C504F501C505F572
:1000100002C506F5076A03C508F50001F5C409F530
:10002000F6C40AF5F7C40BF5F8C40CF5A1AE1CEF45
:1000300000F0B1BE2EEF00F009C5F5F40AC5F6F4E4
:100040000BC5F7F40CC5F8F404C500F505C501F5BA
:1000500006C502F5078E08C503F51100000103016E
:100060001AA901D0196B070E186FCFB60ED01D520A
:100070000CE0CFA405D01B3C01D001D01B2A03D03B
:100080001B5201E01B061D6A03D01D6ACFB61D2A54
:10009000CFB80AD01E5208E01C5202E01C6A02D0FF
:1000A000010E1C6E1E6A03D01E6ACFB81E2AB19EB6
:1000B00000011CEF00F04F5645522D562020000045
:1000C00025352E33664120200000204F5645522D05
:1000D0004920000025342E3266204F464600050E8A
:1000E000EA6E270EE96EEF500EE0140E016E006A04
:1000F000002EFED7012EFBD7BF0E006E002EFED7BE
:1001000000D0EF2EF2D71200FF0EC66EC76EC86E7B
:1001100004010969C89CC89EC790C792C898C89A2C
:10012000A00E00017F6F080E0301F56FF66B1F0E26
:10013000FA6FEF6B100EEE6FE76B840EF36F000E2D
:10014000F86F030E0401006F000E086F106F206F30
:1001500000010EEF04F037A802D0C08801D0C0988B
:1001600037A602D0BF8201D0BF9237A402D0BF8091
:1001700001D0BF9037A202D0C08E01D0C09E37A060
:1001800002D0C08C01D0C09C1200C08A00D0C09A9E
:1001900000D01200640E276EA2DF030E376EDBDF85
:1001A000F4DF050E276E9BDF030E376ED4DFEDDF25
:1001B000010E276E94DF030E376ECDDFE6DF010EF2
:1001C000276E8DDF020E376EC6DFDFDF010E276E72
:1001D00086DF020E376EBFDFD8DF010E276E7FDFAE
:1001E0000E0E376EB8DFD1DF010E276E78DF376A6B
:1001F000B2DFCBDF010E276E72DF080E376EABDF8A
:10020000C4DF010E276E6BDF376AA5DFBEDF010E8C
:10021000276E65DF0C0E376E9EDFB7DF010E276E8F
:100220005EDF376A98DFB1DF010E276E58DF060EFA
:10023000376E91DFAADF010E276E51DF376A8BDF41
:10024000A4DF010E276E4BDF010E376E84DF9DDFCA
:10025000020E276E44DF12EF04F0376A7CDF95DF71
:10026000020E376E78DF91DF020E276E38DF13EF54
:1002700004F00301F38100002A90F3A12A802AB040
:1002800004D02A90F3A12A80FAD7F3B1FED7EBC3AA
:100290002CF5EAC32BF52BC501F52CC502F50001A1
:1002A00012000301EC6BD50E006E002EFED7286AFB
:1002B000276A296A29500F080BE30001DADF02C51B
:1002C00003F50150272602502822292A0301F2D7DC
:1002D0002832273228322732283227322832273252
:1002E0000F0E2816281627C501F528C502F50001AE
:1002F00022EF04F02B38006E0F0E001600500F0B8B
:100300002D6E2B500F0B2C6E2DC537F524DF3DDFE6
:10031000D50E006E002EFED72CC537F51CDF35DF5D
:10032000D50E006E002EFED7AFEF01F02850000A68
:1003300007E0010A06E0030A07E0010A08E00AD024
:1003400009D0400E272606D0140E272603D0540EBF
:10035000272600D0800E27242A6E2B6ECBD71200C2
:100360008E0E006E28C501F527C502F5036A0152FD
:1003700009E102C501F5026A080E005E015202E1C0
:10038000006A08D0D89001BE04D0023601360006BB
:10039000F9D7019E12003450D8B471D0006E385095
:1003A000D8B46DD0002604E3810E002668E204D0A4
:1003B0007F0E005E64E363E035C53CF539503C1ABE
:1003C000358E398E37503B02F4C43EF536503A0232
:1003D000F4C403F5F3C43DF53B02F3503E26F4505C
:1003E0003D22000E032237503A02F3503E26F450CD
:1003F0003D22000E026A0322022235503B02F350D6
:100400003D26F4500322000E022235503A02F350EA
:100410000326F4500222000E016A012237503902ED
:10042000F3503D26F4500322000E022201223650E2
:100430003902F3500326F4500222000E01223550F7
:100440003902F3500226F4500122002A01BE05D0E1
:100450003D360336023601360006000E3DAE0AD0A8
:10046000032A02220122015005E1025003E1035058
:1004700001E1002A3CBE018E3CAE019E04D0006A20
:10048000016A026A036A12003450B608346E036AC5
:1004900035C538F5358ED89035323632373203329D
:1004A000023201320032342EF6D738AE0BD0001EA5
:1004B000011E021E031E002AD8B4012AD8B4022A43
:1004C000D8B4032AE9EF02F0D8B204D0050EEA6EE0
:1004D0003C0EE96E006A016A026A036A3C6A3D6A80
:1004E0003E6A3F6A3B503A10391038102CE0200E1B
:1004F000406ED89034363536363637363C363D3653
:100500003E363F363B503F5C08E13A503E5C05E1E9
:1005100039503D5C02E138503C5C0FE338503C5EA2
:100520003950D8A0393C3D5E3A50D8A03A3C3E5EA6
:100530003B50D8A03B3C3F5ED880003601360236A7
:100540000336402ED6D73CC5EFF43DC5ECF43EC58E
:10055000ECF43FC5ECF412003438356E0F0E35164E
:100560003416100E3524366E376EF5DD0EDE100EA5
:100570003424366E376EEFDD08DED50E006E002EA9
:10058000FED71200E9502C6E2B502E6E19E02AC5B2
:1005900037F529C536F528C535F527C534F53B6A45
:1005A0003A6A200E396E820E386EF5DE03C52AF5E2
:1005B00002C529F501C528F500C527F52E2EE7D778
:1005C0002AC537F529C536F528C535F527C534F5CB
:1005D0005BD703C52AF502C529F501C528F500C575
:1005E00027F52AAE0DD02C062C8A271E281E291E80
:1005F0002A1E272AD8B4282AD8B4292AD8B42A2AC5
:100600003B0E336E9A0E326ECA0E316E306A0A0E8F
:100610002E6E2B50D8B42C2AD882050EEA6E270EE7
:10062000E96E2AC537F529C536F528C535F527C53C
:1006300034F533C53BF532C53AF531C539F530C52A
:1006400038F542DF015000520FE12B282E5C0CE000
:100650002C500CE00F0B2E5C01E037E22CBE35D0A5
:100660002CBC04D0200E2DD0200E2C162CAA0CD081
:100670002C9A2B50D8A42C0600502C6E2D0E346EC4
:100680006BDF2C50006E2C6A2B502E5C0AE1005060
:100690002C6E2E0E346E60DF2C50006E200E2C1649
:1006A000000E300E2CAA0DD02C9A2B50D8A42C065C
:1006B00000502C6E2D0E346E4FDF2C50006E2C6AC5
:1006C000300E002600C534F547DFD89233C537F524
:1006D00032C536F531C535F530C534F53B6A3A6A71
:1006E000396A0A0E386EF0DE03C533F502C532F5FD
:1006F00001C531F500C530F52E2E8ED71200090048
:10070000F55210E0F6C427F5F7C428F5F8C429F52A
:10071000F5C434F521DF27C5F6F428C5F7F429C55B
:10072000F8F4EDD71200010E0301EC6FD50E006E48
:10073000002EFED7286A276A296A29500F080BE382
:10074000000197DD02C503F501502726025028223B
:10075000292A0301F2D728322732283227322832B9
:100760002732283227320F0E2816281627C501F502
:1007700028C502F5000178EF04F00900F6C428F559
:10078000F7C429F5F8C42AF5F5C434F5E5DE28C523
:10079000F6F429C5F7F42AC5F8F4272EEED712008F
:1007A000F86AD69A078EB06BAF6BB36B080EB16F59
:1007B000600EAD6F1B6A1C6A206A1F6A0401006B21
:1007C000086B106B206B0001716B726B736B706B3D
:1007D000756B766B776B746B010E1D6E1E6EB06B56
:1007E000AF6BB36B030EB16F600EAD6F280E276E4B
:1007F00076DCB06BAF6BB36B050EB16F600EAD6F97
:10080000280E276E6CDCB06BAF6BB36B080EB16F4C
:10081000600EAD6F280E276E62DC76D4640E276EF4
:100820005EDCB8D41AD5800E03011A6F460E1B6F1A
:100830001AA901D0196B070E186FA18EC00ED6121F
:1008400000012FD502C526F501C525F5276A286ABE
:100850006DDD253C03D026500F083AE026C528F56B
:1008600025C527F57DDD03C524F502C523F501C5A2
:1008700022F500C521F524C537F523C536F522C577
:1008800035F521C534F5B10E3B6E470E3A6E7A0E42
:10089000396E760E386E7FDD03C524F502C523F56B
:1008A00001C522F500C521F5050EE96E24C52AF51E
:1008B00023C529F522C528F521C527F5030E2B6E82
:1008C00061DE560E346E48DE200E346E45DE07D0F3
:1008D000B60EF66E000EF76E000EF86E10DF276A89
:1008E000010E286E23DD1C5251E01BC57DF01BD785
:1008F00002C526F501C525F5253C03D026500F0875
:100900003DE026C528F525C527F52ADD03C524F5D4
:1009100002C523F501C522F500C521F524C537F52B
:1009200023C536F522C535F521C534F5F60E3B6EE7
:10093000CF0E3A6E530E396E730E386E2CDD03C532
:1009400024F502C523F501C522F500C521F5040EE5
:10095000E96E24C52AF523C529F522C528F521C548
:1009600027F5030E2B6E0EDEC50EF66E000EF76E2B
:10097000000EF86E030E276E00DF07D0CA0EF66E6B
:10098000000EF76E000EF86EBADE3CD07D6B286A62
:100990001BC527F5E5DC03C524F502C523F501C514
:1009A00022F500C521F524C537F523C536F522C546
:1009B00035F521C534F5A10E3B6EA00E3A6E200E22
:1009C000396E770E386EE7DC03C524F502C523F5D2
:1009D00001C522F500C521F5030EE96E24C52AF5EF
:1009E00023C529F522C528F521C527F5020E2B6E52
:1009F000C9DDD90EF66E000EF76E000EF86E040E0D
:080A0000276EBBDE1ED70300C8
:020000040030CA
:0A0000008CFF36DF9FFFFFFFFFFFBC
:00000001FF
